:10000000B8EF17F000000000DAEF16F00000000073
:0C001000000000000000000090EF1CF059
:10001C001E0E0F014D6F100E0001766F040E776FE0
:10002C0076C0E1FF77C0E2FFE69E76C0E1FF77C0C5
:10003C00E2FFE69C040E7625E16E000E7721E26E5F
:10004C00E68C180E8A6F040E8B6F8AC0E1FF8BC092
:10005C00E2FFE69E8AC0E1FF8BC0E2FFE69C040E45
:10006C008A25E16E000E8B21E26EE68C020E76255F
:10007C00E16E000E7721E26E75C2E6FF76C2E6FFF6
:10008C00010E7625E16E000E7721E26E400EE66ED3
:10009C0076C0E9FF77C0EAFFEECF00F076C0E1FF53
:1000AC0077C0E2FF400E0014E66E76C0E9FF77C021
:1000BC00EAFFEECF00F076C0E1FF77C0E2FF880EDA
:1000CC000010E66E76C07AF277C07BF2040E7619D9
:0800DC00006E00C076F0120076
:1000E4000B6A0A6A096A00500402F4CF09F0F3CFDC
:1000F40008F001500502F4CF0BF0F3CF0AF00050E2
:100104000502F3500926F4500A22E86A0B22015032
:100114000402F3500926F4500A22E86A0B2208C0AC
:1001240000F009C001F00AC002F00BC003F0120095
:1001340004012051800AD8A478D0C00E02016B6F4C
:1001440069D00201D00E006E3E0E016E000E026EEA
:1001540000C068F201C069F202C06AF2120E6C6F4C
:10016400000E6D6F62D00201030E006E000E016E70
:1001740022C404F0000E056EB3DF8E0E0024E96E77
:10018400030E0120EA6EEECF68F2EECF69F2EECFF5
:100194006AF2020E6825F66E000E6921F76E000EF3
:1001A4006A21F86E0900F5CF00F00900F5CF01F0DF
:1001B40000C06CF201C06DF238D00401225102017A
:1001C4005A5D23E3030E006E000E016E22C404F098
:1001D400000E056E85DF7E0E0024E96E030E0120FD
:1001E400EA6EEECF68F2EECF69F2EECF6AF268C241
:1001F400F6FF69C2F7FF6AC2F8FF0900F5CF00F005
:1002040000C06CF2000E6D6F01D06B6B0ED002015A
:100214006B6B0BD004012351010A93E02351020AB2
:0C022400A2E02351030AC9E0F2D7120047
:10023000000E02016D5D02E1080E6C5D11E26CC200
:1002400003F06DC204F000018F51000A03E1010EBA
:100250008F6F05D08F51010A02E1020E8F6F04D01B
:10026000080E036E000E046E000188C0E1FF89C015
:10027000E2FFE69288C0E1FF89C0E2FFE69088C015
:10028000E9FF89C0EAFFEECF00F088C0E1FF89C036
:10029000E2FF04500010E66E010E8825E16E000EAC
:1002A0008921E26E03C0E6FF035002016C5D006E1F
:1002B00004506D59016E00C06CF201C06DF2280E41
:1002C0006E6F040E6F6F6BB12FD0035004102BE0D4
:1002D00068C2F6FF69C2F7FF6AC2F8FF0900F5CFEE
:1002E00000F06EC2E1FF6FC2E2FF00C0E6FF6E4B9E
:1002F0006F2B010E6825006E000E6921016E000E45
:100300006A21026E00C068F201C069F202C06AF29E
:10031000010E035C006E000E0458016E00C003F075
:1003200001C004F0D2D724D00350041021E068C2E9
:10033000E9FF69C2EAFF6EC2E1FF6FC2E2FFEECFE2
:10034000E6FF6E4B6F2B010E6825006E000E6921D3
:10035000016E00C068F201C069F2010E035C006E1C
:10036000000E0458016E00C003F001C004F0DCD799
:02037000120079
:1003720020C401F01F0E01160150010A01E094D0C1
:1003820004012451000A01E08FD02151060A42E102
:1003920037D002015851010A17E1950E006E3B0E4B
:1003A200016E000E026E120E0026000E01220222C3
:1003B20000C068F201C069F202C06AF2090E6C6FF5
:1003C200000E6D6FC00E6B6F25D002015851010AED
:1003D20012E1720E006E3C0E016E000E026E00C043
:1003E20068F201C069F202C06AF2210E6C6F000E5F
:1003F2006D6FC00E6B6F0ED00201800E6B6F0AD054
:1004020004012351210AC5E02351220ADEE02351CF
:10041200230AF2E020C401F0600E0116050E006E00
:10042200005004E00132019EFF0FFBD70150010A88
:1004320001E03AD026D038D037D0770E0201686F6B
:10044200020E696F010E6C6F000E6D6FC10E6B6F45
:100452002BD00201800E6B6F23C477F225D00201EC
:10046200700E686F020E696F010E6C6F000E6D6F79
:10047200810E6B6F19D00201800E6B6F22C470F275
:1004820013D004012151010AD6E02151090AD4E016
:100492002151020AD2E021510A0ADBE02151030A6A
:0A04A200DEE021510B0AE7E0120032
:1004AC0004012251010A13E120C401F01F0E0116B0
:1004BC000150000A0CE102016B8F04012151030A67
:1004CC0004E1010E0201726F02D00201726B040191
:1004DC002251000AD8A48DD020C401F01F0E0116A1
:1004EC000150020AD8A485D024C401F00F0E0116C5
:1004FC000150000AD8B47DD002016B8F040124BFD7
:10050C0016D024C403F00F0E031603C000F0000E27
:10051C00016E003600900136740E0024E96E000E58
:10052C000120EA6EEECF04F0EECF05F015D024C416
:10053C0003F00F0E031603C000F0000E016E003620
:10054C0000900136880E0024E96E000E0120EA6E40
:10055C00EECF04F0EECF05F02151030A07E104C001
:10056C00E1FF05C0E2FF840EE66E43D024C400F028
:10057C000F0E00164C0E026E0F0E036E005002266C
:10058C00D8B0032A02C0E9FF03C0EAFFFE0EEE1446
:10059C00006EEECF01F0FF0E011602C0E1FF03C0AA
:1005AC00E2FF00C0E6FF01C0E6FF24AF11D004C09B
:1005BC00E1FF05C0E2FFE66A040E0418006E00C0FD
:1005CC0004F004C0E1FF05C0E2FF400EE66E11D05E
:1005DC0004C0E1FF05C0E2FF880EE66E040E0418AD
:1005EC00006E00C004F004C0E1FF05C0E2FFC80EBD
:0405FC00E66E120095
:1006000002016B8F0F014D6B0201716B22C458F216
:100610005851000A04E1100E0001856F04D000015A
:08062000200E856FFBDC1200C7
:100628000401286B296B4AD002016B8F04012881D1
:1006380002017251010A02E10401288354D0020127
:100648006B8F51D002016B8F040124BF16D024C4D4
:1006580003F00F0E031603C000F0000E016E003603
:1006680000900136740E0024E96E000E0120EA6E37
:10067800EECF04F0EECF05F015D024C403F00F0E32
:10068800031603C000F0000E016E0036009001361C
:10069800880E0024E96E000E0120EA6EEECF04F009
:1006A800EECF05F004C0E9FF05C0EAFFEECF01F088
:1006B80001A403D00401010E286F15D020C401F055
:1006C8001F0E01160150000AAFE020C401F01F0EF2
:1006D80001160150010AB3E020C401F01F0E0116F3
:1006E8000150020AAFE002016BAF07D0280E686F15
:0C06F800040E696F6B81020E6C6F120023
:10070400160E0F015F6F9F0E5D6F3B0E5C6F120044
:10071400010E00016D25E96E000E6E21EA6EEECF2A
:1007240000F000C002F0000E0201635D02E102501D
:10073400625D03E262C202F00AD00250625D006EA2
:10074400000E6359016E00C062F201C063F2036AD5
:100754000250035C1CE2280EE96E040EEA6E03509C
:10076400E926D8B0EA2AEECF00F05FC2E1FF60C20A
:10077400E2FF00C0E6FF010E5F25006E000E60215F
:10078400016E00C05FF201C060F2032AE1D7000EDF
:10079400006E6351005C02E16251000829E2010E1F
:1007A40000017125E16E000E7221E26E080EE66E04
:1007B400020E7125E16E000E7221E26E280EE66EC5
:1007C400040EE66E6DC0E9FF6EC0EAFFEECF00F0E6
:1007D40000BC07D071C0E1FF72C0E2FFC80EE66E34
:1007E40006D071C0E1FF72C0E2FF880EE66E1BD036
:1007F4000001010E7125E16E000E7221E26E080EF9
:10080400E66E020E7125E16E000E7221E26E200E7C
:10081400E66E040EE66E71C0E1FF72C0E2FF840E64
:08082400E66E0201619F120063
:10082C00659802016BBF4BD061AF29D0020E00015D
:10083C008C6F010E8825E16E000E8921E26EE66A4E
:10084C0088C0E1FF89C0E2FFC80EE66E010E71257B
:10085C00E16E000E7221E26E080EE66E020E71253C
:10086C00E16E000E7221E26E280EE66E040EE66E4C
:10087C0071C0E1FF72C0E2FFC80EE66E1FD000012E
:10088C00010E7125E16E000E7221E26E080EE66E0D
:10089C00020E7125E16E000E7221E26E200EE66EE4
:1008AC00040EE66E71C0E1FF72C0E2FF8C0EE66EC4
:1008BC0088C0E1FF89C0E2FF840EE66E88D0020199
:1008CC0061BF85D0040120AF5AD002016D510401E3
:1008DC00275D04E102016C510401265D04E226C48B
:1008EC006CF227C46DF29EDC010E00018C6F010EC0
:1008FC007125E16E000E7221E26E080EE66E020E9C
:10090C007125E16E000E7221E26E200EE66E040E71
:10091C00E66E71C0E1FF72C0E2FF800EE66E02016E
:10092C00786B010E00016D25E16E000E6E21E26EFA
:10093C00080EE66E020E6D25E16E000E6E21E26E63
:10094C00200EE66E040EE66E6DC0E1FF6EC0E2FF97
:10095C00840EE66E010E0201786F020E00018825EE
:10096C00E16E000E8921E26E280EE66E040EE66E34
:10097C0088C0E1FF89C0E2FFC80EE66E28D00001F6
:10098C00020E8C6F010E8825E16E000E8921E26E3D
:10099C00E66A88C0E1FF89C0E2FFC80EE66E010E70
:1009AC007125E16E000E7221E26E080EE66E020EEB
:1009BC007125E16E000E7221E26E280EE66E040EB9
:1009CC00E66E71C0E1FF72C0E2FFC80EE66E120067
:1009DC0000018C6B88C0E1FF89C0E2FFE66A040E5F
:1009EC008819E16E89C0E2FF000EE21AE66A020184
:0809FC0061AF01D0619F120000
:100A040020C401F0600E0116050E006E005004E0D3
:100A14000132019EFF0FFBD70150000A01E060D0B4
:100A24003CD002016B8F080E0001856F59D09AECFF
:100A340000F056D0E3DD54D0580E0201686F020E68
:100A4400696F6B81010E6C6F6B8F4AD0EBDD48D000
:100A54002BDD46D0710E006E020E016E040124518E
:100A64000026D8B0012A00C068F201C069F2020170
:100A74006B81010E6C6F6B8F33D002016B8F710E23
:100A8400E16E020EE26E04012451E126D8B0E22A9E
:100A940022C4E6FF25D024D023D004012151050A25
:100AA400C0E02151060AC3E02151090AC3E02151E3
:100AB400080AC2E02151000AC9E02151010AC8E034
:100AC4002151030AC5E021510A0AC4E021510B0A4D
:100AD400D4E02151070ADFE021510C0ADDE0DCD724
:020AE4001200FE
:0A0AE6000201595301E042DC120046
:100AF000950E03018E6F3B0E8F6F000E906F2F0EC1
:100B00007E6F410E7F6F000E806F500E816F3C0E26
:100B1000826F000E836FB30E846F3C0E856F000EE4
:040B2000866F1200CA
:100B240065920F015C9562A403D0FB0E6216FBD79D
:020B34001200AD
:100B36000F014CA119D06DC0E9FF6EC0EAFFEECFE0
:100B460001F00150800A0FE188C0E9FF89C0EAFF81
:100B5600EECF01F00150840A06E16DC0E1FF6EC0E0
:0E0B6600E2FF8C0EE66E4C91DF0E621612005E
:100B7400040E00018819006E00C088F08551080A2F
:100B84000DE122C45EFF0F015E51000804E2100E65
:100B94000001856F03D00001040E856F8C51010A9A
:100BA4003CE1020E8825E16E000E8921E26E280EDA
:100BB400E66E040EE66E18EC01F000018F51020A95
:100BC40007E188C0E1FF89C0E2FF840EE66E24D00D
:100BD400040E8819006E00C088F088C0E9FF89C03F
:100BE400EAFFEECF00F000BC0CD0040E8819006EB2
:100BF40000C088F088C0E1FF89C0E2FFC80EE66E3D
:100C04000BD0040E8819006E00C088F088C0E1FF84
:0E0C140089C0E2FF880EE66E01D0DEDE12001F
:0C0C22000F015C85EF0E62166582120067
:100C2E006DB409D01F0E6B14016E0150000A03E162
:0A0C3E00010E006E01D0006A1200E2
:100C480053DF02017A6B7B6B7C6B7D6B636A626A34
:100C580055DD658C5E6B4D6B659C02015B6B5C6B57
:100C6800000E5C5D02E1080E5B5D17E25BC200F0FE
:100C78005CC201F000360090013600360090013663
:100C8800000E0024E16E040E0120E26EE66AE66AB8
:100C9800E66AE66A5B4B5C2BE3D7160E0F014C6FD6
:100CA80062A603D0F70E6216FBD702016B6B616B6D
:100CB800626B636B6598080E0001886F040E896F7C
:0A0CC8000201586B0001856B120059
:040CD200A1981200D3
:100CD60000018C51020A02E11ADD20D07CDE785137
:100CE600000A1AE1010E00017125E16E000E722163
:100CF600E26E080EE66E020E7125E16E000E72219E
:100D0600E26E200EE66E040EE66E71C0E1FF72C062
:0E0D1600E2FF8C0EE66E02D00201786B120036
:100D240088C0E9FF89C0EAFFEECF00F000AE05D02D
:100D340088C0E1FF89C0E2FFE66A00018F6B8C6B1B
:100D440002016C6B6D6B6B6B5BDECBDE6DDD1200D9
:0E0D5400ADB202D00000FCD7C4C3AEFF120047
:100D620000018551000A0BE1656A0F015C6BC9DC69
:100D720065B602D06586FCD7010E0001856F8551EC
:100D8200010A0AE165BA08D0626A0F015C6B5C81F4
:100D92005C89020E0001856F62A406D00F015CA57A
:100DA20003D0FB0E6216BDDE65A202D091DFE0D059
:100DB20062A019D00F015CA116D045DF040E856F29
:100DC200200E0401026F040E036F080E016F000E65
:100DD2000015006E00C000F48C0E0011006E00C001
:100DE20000F4FE0E621662A806D00F015CA903D0C1
:100DF20017DFEF0E621662AC05D00F015CAD02D0B8
:100E0200BF0E621662AA04D00F015CAB01D092DE63
:100E120062A204D00F015CA301D0636A040E000138
:100E2200855D02E255DFA4D00F015CA7A0D00301CB
:100E3200C56B040EC55DD8B09AD062A694D064CFBB
:100E420081F0F70E6216780E00018115016E0150D5
:100E5200000AD8A487D0FD0E8115016E026AFF0E2A
:100E62000216000E021802E1000E01186CE17E0E5D
:100E72008115016E01C003F00332039E03C000F02E
:100E8200000E016E003600900136003600900136E9
:100E9200000E0024026E040E0120036E02C06DF0EB
:100EA20003C06EF002C071F003C072F0040E71193B
:100EB200006E00C071F002C0E9FF03C0EAFFEECF8E
:100EC20000F000C001F03C0E01160132019E013219
:100ED200019E01500D0A35E1020E6D25E96E000EEC
:100EE2006E21EA6EEECF01F0EECF02F00250040A5C
:100EF20002E1280E011823E1020E6D25E16E000EBB
:100F02006E21E26E200EE66E040EE66E0301C46BE5
:100F1200080EC45D14E2200EE16E040EE26EC451AE
:100F2200E126D8B0E22A280EE96E040EEA6EC45118
:100F3200E926D8B0EA2AEECFE6FFC42BE9D7F1DEE4
:100F420001D0C8DE0ED0FD0E00018115016E026ACD
:100F5200FF0E0216000E021802E1040E011801E152
:100F620008DE00D001D003D00301C52B62D7B0DE6A
:020F720012006B
:100F74000301C551000A12E0C4C300F0000E016E63
:100F8400003600900136880E0024E96E000E012020
:100F9400EA6EEECF04F0EECF05F011D0C4C300F03A
:100FA400000E016E003600900136740E0024E96EC6
:100FB400000E0120EA6EEECF04F0EECF05F0020E33
:100FC4000424E16E000E0520E26EC6C3E6FFC7C32B
:100FD400E6FF010E0424E16E000E0520E26EC8C394
:100FE400E6FF04C0E9FF05C0EAFFEECF00F004C04D
:100FF400E1FF05C0E2FF400E0014E66E04C0E9FF05
:1010040005C0EAFFEECF00F004C0E1FF05C0E2FF37
:10101400880E0010E66EC551000A1BE0C4C300F040
:10102400000E016E003600900136880E0024026E18
:10103400000E0120036E02C0E9FF03C0EAFF040EA4
:10104400EE18006E02C0E1FF03C0E2FF00C0E6FF3D
:101054001AD0C4C300F0000E016E003600900136B1
:10106400740E0024026E000E0120036E02C0E9FF1C
:1010740003C0EAFF040EEE18006E02C0E1FF03C0D5
:10108400E2FF00C0E6FF04C000F005C001F012005A
:10109400000E0301C51902E1000EC41902E1016A40
:1010A4000AD0C4C3E9FFC5C3EAFFEECF00F0000EC7
:0C10B40000BE010E016E01C000F0120031
:1010C0000301C46BC56BC551120802E1C4518E08FF
:1010D00008E3ADDD005201E004D00301C44BC52B91
:1010E000F2D70301120EC55D02E18F0EC45D03E36A
:1010F0007B0E006E05D06B806BA001D0FDD7006A1F
:021100001200DB
:041102006B841200E8
:10110600A49EC4C36FFF6DA401D0FDD7A4BE01D0B9
:10111600FDD76BBC02D0006A03D06B84020E006E52
:021126001200B5
:10112800C6C3F6FFC7C3F7FFC8C3F8FF0900F5CF6A
:1011380000F0005218E0C6C3F6FFC7C3F7FFC8C3E4
:10114800F8FF0900F5CF00F0C4C3E1FFC5C3E2FF13
:1011580000C0E6FF0301C44BC52B010EC627000ED5
:10116800C723C823DDD7C4C3E1FFC5C3E2FFE66ACE
:02117800120063
:0A117A006B826BA201D0FDD71200BA
:10118400D00E006E3E0E016E000E026E0E0E002496
:10119400F66E000E0120F76E000E0220F86E0900B4
:1011A400F5CF03F003C004F00F0E0024F66E000E1A
:1011B4000120F76E000E0220F86E0900F5CF01F051
:1011C4000150035C12E2D00E006E3E0E016E000E62
:1011D400026E0F0E0024F66E000E0120F76E000E54
:1011E4000220F86E0900F5CF04F0D00E006E3E0E1A
:1011F400016E000E026E100E0024F66E000E012029
:10120400F76E000E0220F86E0900F5CF01F00150D0
:10121400045C12E2D00E006E3E0E016E000E026EF1
:10122400100E0024F66E000E0120F76E000E022050
:0E123400F86E0900F5CF04F004C000F01200BF
:0A124200D08EA288A088F28E120060
:10124C003C0E7B6EAF0E7A6E02015D6B5E6B79802D
:08125C00A192A292A0821200EF
:101264000301A96BAA6BAB6B020EA625F66E000EEA
:10127400A721F76E000EA821F86E0900F5CF05F03E
:10128400030EA625F66E000EA721F76E000EA82108
:10129400F86E0900F5CF00F000C003F0000E046EF4
:1012A40003C001F0006A05500024066E000E012000
:1012B400076EA6C308F0A7C309F0A8C30AF0010E7D
:1012C4000824F66E000E0920F76E000E0A20F86E50
:1012D4000900F5CF01F00150020A1BE1060E0824B3
:1012E400F66E000E0920F76E000E0A20F86E090053
:1012F400F5CF01F00150A95D0CE2060E0824F66E4C
:10130400000E0920F76E000E0A20F86E0900F5CFD2
:10131400A9F3010E0824F66E000E0920F76E000EE4
:101324000A20F86E0900F5CF01F00150040A1BE110
:10133400080E0824F66E000E0920F76E000E0A202F
:10134400F86E0900F5CF01F00150A95D0CE2080E1A
:101354000824F66E000E0920F76E000E0A20F86EBF
:101364000900F5CFA9F308C0F6FF09C0F7FF0AC0CA
:10137400F8FF0900F5CF00F00050AA25016E000E19
:10138400AB21026E01C0AAF302C0ABF30750025CAA
:1013940002E10650015C01E30FD008C0F6FF09C06A
:1013A400F7FF0AC0F8FF0900F5CF00F00050082647
:0E13B400000E09220A2283D7A9C300F01200FE
:1013C2007EDE8DC3C4F39EDE0301C46B9BDE020E80
:1013D2000301C46F97DE0BD0800E0301C46F92DE4F
:1013E20014D0C00E0301C46F8DDE0FD00ED0000EDC
:1013F2000301A71902E1010EA619EEE0000EA719DA
:1014020002E1020EA619EDE0F1D7B6DE8DC3C4F3F8
:1014120079DE400E0301C46F75DE0001826B836BBF
:10142200000E835D02E17351825D08E2A00E0301AA
:10143200C46F68DE0001824B832BF2D79DDE8DC321
:10144200C4F360DE0301C46B5DDE0BD0800E0301CA
:10145200C46F58DE14D0C00E0301C46F53DE0FD028
:101462000ED0000E0301A71902E1010EA619EEE04B
:10147200000EA71902E1020EA619EDE0F1D740DE37
:02148200120056
:101484000301A96BA6C3E9FFA7C3EAFFEECFA8F344
:10149400A851000A0EE0A8C3C4F35ADC0301A92B27
:1014A400A951A625E96E000EA721EA6EEECFA8F396
:0414B400EFD712005C
:0E14B800A8B202D00000FCD7A6C3A9FF120004
:1014C600FCDD8DC3C4F31CDE0301C46B19DE000E04
:1014D600006E0301A951005C03E1A8510001735D90
:1014E60005E273C0A8F3000E0301A96F0FD0030134
:1014F600A851800FC46FC40703DE16D00301A8519C
:10150600C00FC46FC407FCDD0FD00ED0000E030160
:10151600A71902E1010EA619EAE0000EA71902E1D9
:10152600020EA619EBE0F1D725DE8DC3C4F3E8DD84
:10153600400E0301C46FE4DDA8C3ACF3A9C3ADF349
:10154600AAC3E9FFABC3EAFFEE521AE0AAC3D9FF6A
:10155600ABC3DAFFDE50800F0301C46FD1DD030198
:10156600AA4BAB2BAC4BAD2B800E006E800EAD198B
:10157600005C03E1AC510001735D01E201D0E0D7EC
:04158600BDDD1200B5
:10158A00A6C3F6FFA7C3F7FFA8C3F8FF0900F5CF64
:10159A0000F0005212E0A6C3F6FFA7C3F7FFA8C3E4
:1015AA00F8FF0900F5CFC4F3AAEC06F0010E030117
:0C15BA00A627000EA723A823E3D71200E9
:1015C600200E0001855D03E365B201D002D0006AFA
:1015D6004AD07CC2C4F37DC2C5F359DD005242E154
:1015E600A9C3C4F3010EC56FA6C3C6F3A7C3C7F349
:1015F600A8C3C8F3BCDC00C07CF201C07DF20201C6
:10160600546B556B566B576B7CC2C4F37DC2C5F3E6
:101616003EDD005210E0010E016E0150000A02E1AB
:10162600B1EC06F00201545155115611571102E062
:10163600006A19D0E9D702017CC2AAF37DC2ABF3D6
:10164600000E7D1902E1000E7C190AE0010E03016D
:10165600AA25E96E000EAB21EA6EEECF00F003D0AC
:08166600006A01D0006A1200C5
:10166E000D0E0301C46FAAEC06F00A0E0301C46F3F
:06167E00AAEC06F01200C8
:101684001DDD8DC3C4F33DDD0301C46B3ADD800E63
:10169400006E800E0301A919005C03E1A85100014A
:1016A400735D05E273C0A8F3000E0301A96F0FD0A8
:1016B4000301A851800FC46FC40723DD16D00301B2
:1016C400A851C00FC46FC4071CDD0FD00ED0000E8C
:1016D4000301A71902E1010EA619EAE0000EA719F9
:1016E40002E1020EA619EBE0F1D745DD8DC3C4F388
:1016F40008DD400E0301C46F04DD0301AA51800F0D
:08170400C46FFFDCFCDC1200E5
:10170C00086A080E0C6E003408360450085ED8B017
:0E171C0002D00826D89000360C2EF5D7120009
:10172A00AD0E0301C46F030EC56FAAC3C6F3ABC3E4
:10173A00C7F3ACC3C8F3F3DCBEDC8DC3C4F3DEDC91
:10174A000301C46BDBDC000E006E0301A951005CCF
:10175A0003E1A8510001735D05E273C0A8F3000E0E
:10176A000301A96F0FD00301A851800FC46FC407EA
:10177A00C5DC16D00301A851C00FC46FC407BEDC74
:10178A000FD00ED0000E0301A71902E1010EA6190F
:10179A00EAE0000EA71902E1020EA619EBE0F1D762
:1017AA00E7DC8DC3C4F3AADC400E0301C46FA6DCD8
:1017BA00A8C3C2F3A9C3C3F3AAC3F6FFABC3F7FF17
:1017CA00ACC3F8FF0900F5CF00F0005222E0AAC32B
:1017DA00F6FFABC3F7FFACC3F8FF0900F5CF00F083
:1017EA000050800F0301C46F89DC010E0301AA2790
:1017FA00000EAB23AC23C24BC32B800E006E800EAF
:10180A00C319005C03E1C2510001735D01E201D01A
:06181A00D3D772DC1200BE
:0E182000570E0D6E0D2EFED7000000001200B8
:10182E00AADC00C0A0F3950E0301A66F3B0EA76FB6
:10183E00000EA86F10DD00C0A1F3A051005C03E202
:0C184E00A0C300F002D0A1C300F0120003
:10185A00A0C3A6F3A1C3A7F3A2C3A8F3010E030171
:06186A00A96FACDE1200C4
:101870000301A36B030EA35D0AE2A351A125E16E50
:10188000000EA221E26E200EE66EA32BF3D7A35129
:10189000A125E16E000EA221E26EE66AA307A35124
:1018A000A125A46F000EA221A56F0A0E046EA0C38D
:1018B00000F02CDF08C000F0300E0026A4C3E1FFCA
:1018C000A5C3E2FF00C0E6FF0A0E046EA0C300F04D
:1018D0001DDF00C0A0F30050000A01E102D0A30701
:0418E000DED712003D
:1018E400A0C3F6FFA1C3F7FFA2C3F8FF0900F5CF19
:1018F40000F0005211E0A0C3F6FFA1C3F7FFA2C39A
:10190400F8FF0900F5CFA6F3D5DD010E0301A027EA
:0A191400000EA123A223E4D7120065
:10191E0000016B6B6C6B010E6C5D02E1000E6B5D7A
:10192E000AE2400E6B25E16E010E6C21E26EE66A54
:10193E006B4B6C2BF0D701013C6B3D6B00016B6B5D
:10194E006C6BA4AA02D0AACF78F0786B0201406B20
:06195E00416BA38A120098
:10196400086A096A100E0C6E0134083609360450F0
:10197400085E0550D8A0053C095ED8B007D00450D5
:1019840008260550D8B0053C0926D8900036013603
:061994000C2EEAD7120040
:10199A00A4C301F0A5C302F0010E0301A45F000E67
:1019AA00A55B000E021802E1000E01181FE0A0C399
:1019BA00E9FFA1C3EAFFA2C3D9FFA3C3DAFFEE502E
:1019CA00DE180FE0A0C3E9FFA1C3EAFFA2C3D9FF53
:1019DA00A3C3DAFFDE50EE5C006E016A000E015A04
:1019EA0007D0A04BA12BA24BA32BD2D7006A016A26
:0219FA001200D9
:1019FC0000018551000A0DE1656A0F015C6B82ECF8
:101A0C0003F019DC65B602D06586FCD7010E000127
:041A1C00856F1200C0
:101A2000400E00016F6F010E706F21DEC50E0301C5
:101A3000A66F400EA76F000EA86FA7DD400E030132
:101A4000A66F010EA76F1EDD12DE01014F6B010EA6
:101A50000301A66F000EA76FB4DC010E0301A66F91
:101A6000000EA76F010EA86F000EA96F400EAA6F9F
:101A7000010EAB6F28DD020E0301A66F000EA76FEB
:101A8000010EA86F000EA96F270EAA6F3F0EAB6F55
:101A9000000EAC6F4ADE000E02015E1902E1000E7C
:101AA0005D1921E1524B532B020E0301A66F000E6C
:101AB000A76F090EA86F000EA96F300E0201522504
:101AC0000301AA6FDFDD3D0E0B6EE10E0C6E3F0EC3
:101AD0000D6E0D2EFED70C2EFCD70B2EFAD7000064
:101AE00000008C9801D08C88A40E0301A66F400ED4
:101AF000A76F000EA86F49DD300E020152250301C9
:101B0000C46FAAEC06F0B3DD070E0B6E170E0C6E59
:101B10006A0E0D6E0D2EFED70C2EFCD70B2EFAD7AB
:101B200000000F0E01013E6F000E3F6F26EC09F022
:021B30001200A1
:101B3200540E0301916F0D0E926FC40E936F030E3C
:101B4200946FFF0E00017D6FFF0E7E6F000E7F6FA0
:101B5200000E806FFF0E796FFF0E7A6F000E7B6FA3
:101B6200000E7C6FFF0E676FFF0E686F000E696FCD
:101B7200000E6A6FAD8A900EAC6E948E949C9EAAF3
:0A1B820003D0AFCF00F0FBD7120034
:101B8C0097C304F098C305F095C302F096C303F015
:101B9C0099C300F09AC301F0010E0301995F000E86
:101BAC009A5B005001100FE004C0E9FF05C0EAFF8A
:101BBC0002C0E1FF03C0E2FFEECFE6FF024A032AB8
:101BCC00044A052AE5D795C300F096C301F012002C
:101BDC00B80E0301916F140E926FA60E936F030E45
:101BEC00946FFF0E00017D6FFF0E7E6F000E7F6FF6
:101BFC00000E806FFF0E796FFF0E7A6F000E7B6FF9
:101C0C00000E7C6FFF0E676FFF0E686F000E696F22
:101C1C00000E6A6FA88A900E9C6E98849892A4AA63
:0A1C2C0003D0AACF00F0FBD712008E
:101C3600FBDD00C05AF2010E0201596F95C375F221
:101C460096C376F297C373F298C374F224EC06F047
:0E1C5600010E016E0150010A01E1CDDE120007
:101C6400959A959C8C9A8C9C958A958C6D9E6D9C6E
:061C7400380E6C6E120038
:101C7A00C26A070EC16EC18E95C300F0003600908D
:101C8A00003600900050C212C280C5DDC282C2A2D4
:101C9A0001D0FDD7C4CF01F0006AC3500012000E74
:061CAA000112C2901200BD
:101CB0000900F5CFE6FF0006FBE10106F9E112009D
:101CC00000018551010A09E165BA07D0626A0F0176
:101CD0005C815C89020E0001856F62A407D00F0150
:101CE0005CA504D0FB0E621692EC05F065A203D051
:101CF00069EC06F0E8D062A01AD00F015CA117D001
:101D000024EC06F0040E856F200E0401026F040E11
:101D1000036F080E016F000E0015006E00C000F486
:101D20008C0E0011006E00C000F4FE0E621662A858
:101D300007D00F015CA904D011EC06F0EF0E62167B
:101D400062AC05D00F015CAD02D0BF0E621662AA74
:101D500005D00F015CAB02D09BEC05F062A204D071
:101D60000F015CA301D0636A040E0001855D03E2EC
:101D700069EC06F0A8D00F015CA7A3D00301CA6BE1
:101D8000040ECA5DD8B09DD062A697D064CF81F012
:101D9000F70E6216780E00018115016E0150000ADF
:101DA000D8A48AD0FD0E8115016E026AFF0E0216BC
:101DB000000E021802E1000E01186EE17E0E811580
:101DC000016E01C003F00332039E03C000F0000E59
:101DD000016E003600900136003600900136000E8C
:101DE0000024026E040E0120036E02C06DF003C0D9
:101DF0006EF002C071F003C072F0040E7119006E33
:101E000000C071F002C0E9FF03C0EAFFEECF00F0AE
:101E100000C001F03C0E01160132019E0132019E0C
:101E200001500D0A36E1020E6D25E96E000E6E219D
:101E3000EA6EEECF01F0EECF02F00250040A02E1AA
:101E4000280E011823E1020E6D25E16E000E6E21B1
:101E5000E26E200EE66E040EE66E0301C96B080EFC
:101E6000C95D14E2200EE16E040EE26EC951E12656
:101E7000D8B0E22A280EE96E040EEA6EC951E926AE
:101E8000D8B0EA2AEECFE6FFC92BE9D792EC06F0EC
:101E900002D06BEC06F00FD0FD0E00018115016E33
:101EA000026AFF0E0216000E021802E1040E01186B
:101EB00002E1BAEC05F000D001D003D00301CA2B37
:081EC0005FD769EC06F0120087
:101EC8008C988D981F0E0B6E710E0C6E1E0E0D6E7B
:101ED8000D2EFED70C2EFCD70B2EFAD700008C88BF
:101EE8001F0E0B6E710E0C6E1E0E0D6E0D2EFED794
:101EF8000C2EFCD70B2EFAD700008C988D881F0E5D
:101F08000B6E710E0C6E1E0E0D6E0D2EFED70C2E66
:101F1800FCD70B2EFAD700008C888D981F0E0B6EFD
:101F2800710E0C6E1E0E0D6E0D2EFED70C2EFCD7EC
:0C1F38000B2EFAD700008C988D98120038
:101F440095C304F096C305F004C0E9FF05C0EAFF99
:101F5400EE5203E0044A052AF7D704C002F005C094
:101F640003F0044A052A97C300F098C301F0030163
:101F7400974B982B00C0E9FF01C0EAFF02C0E1FFC4
:101F840003C0E2FFEECFE6FF02C0E9FF03C0EAFFB1
:101F9400EE5201E0E2D795C300F096C301F01200BF
:101FA400FD0EC16EFF0EC26EFF0E926E9294FF0E76
:101FB400936EFF0E956EFF0E946EFF0E986E959CB9
:101FC400958E9986959896988C988D9895949382E9
:021FD4001200F9
:101FD6007E0E03018925E16E020E8A21E26EE66A13
:101FE600876B886B896B8A6B9EAA02D0AFCF79F21A
:0E1FF6000201796B03018B6B8C6BA08A1200C9
:102004000301986B95C3E9FF96C3EAFFEECF97F3FC
:102014009751000A0FE097C3A6F35CEC0AF00301A2
:10202400982B98519525E96E000E9621EA6EEECF15
:0620340097F3EED7120045
:10203A000301996B050E995D0AE299519725E16EA4
:10204A00000E9821E26E200EE66E992BF3D7995175
:10205A009725E16E000E9821E26EE66A990799517A
:10206A0097259A6F000E98219B6F0A0E046E000E38
:10207A00056E95C300F096C301F06FDC08C000F04E
:10208A0009C001F0300E00269AC3E1FF9BC3E2FFAC
:10209A0000C0E6FF0A0E046E000E056E95C300F03E
:1020AA0096C301F05ADC00C095F301C096F3000E06
:1020BA00011802E1000E001801E102D09907CFD7FA
:0220CA00120002
:1020CC0095C304F096C305F0030199519A1124E0CD
:1020DC00010E995F000E9A5B04C002F005C003F07C
:1020EC00044A052A97C300F098C301F0974B982B2C
:1020FC0000C0E9FF01C0EAFF02C0E1FF03C0E2FF3C
:10210C00EECFE6FF02C0E9FF03C0EAFFEECF00F01E
:10211C00005201E101D0D8D799C300F09AC301F065
:10212C00010E995F000E9A5B0050011008E004C08C
:10213C00E1FF05C0E2FFE66A044A052AEDD795C324
:08214C0000F096C301F012003F
:1021540099C300F003019907005228E095C3E9FFF1
:1021640096C3EAFFEE50000A0CE095C3E9FF96C35C
:10217400EAFF97C3D9FF98C3DAFFEE50DE1801E1F6
:102184000FD095C3E9FF96C3EAFF97C3D9FF98C35D
:10219400DAFFDE50EE5C006E016A000E015A08D0D0
:1021A4000301954B962B974B982BD2D7006A016A63
:0221B400120017
:1021B6000D0E0501406F0A0E416F426B400E030182
:1021C600A06F050EA16F400EA26F2DEC0CF0005211
:0621D60001E1F4D7120044
:1021DC00010E0301A66F000EA76F010EA86F000E73
:1021EC00A96F050EAA6F3F0EAB6F000EAC6F95EC8E
:1021FC000BF0020E0301A66F000EA76F010EA86F65
:10220C00000EA96F380EAA6F3F0EAB6F000EAC6FAD
:10221C0095EC0BF01F0E0B6E710E0C6E1E0E0D6EF0
:10222C000D2EFED70C2EFCD70B2EFAD700008C9857
:10223C008D98260E0301A66F410EA76F000EA86F96
:10224C00C5EC0AF0170E0301A06F410EA16F000E32
:10225C00A26F72EC0CF01F0E0B6E710E0C6E1E0E3C
:10226C000D6E0D2EFED70C2EFCD70B2EFAD70000C0
:10227C000201526B536B320E01013E6F000E3F6F29
:10228C0026EC09F0830E0301A66F3E0EA76F000E1D
:10229C00A86FC5EC0AF08FEC0CF0240E0301A66FAE
:1022AC005CEC0AF04E0E0C6EEB0E0D6E0D2EFED786
:1022BC000C2EFCD7240E0301A66F5CEC0AF04E0E1C
:1022CC000C6EEB0E0D6E0D2EFED70C2EFCD7240EC5
:1022DC000301A66F5CEC0AF04E0E0C6EEB0E0D6E4D
:1022EC000D2EFED70C2EFCD7000E0201411902E177
:1022FC00000E40190EE1000E5E1902E1000E5D1990
:10230C0008E1000E01013D5D02E1030E3C5D01E2BE
:10231C00EBD7400E0301A06F010EA16F4E0EA26F02
:10232C00000EA36F030EA46F000EA56FCDEC0CF086
:10233C00000E011802E1000E001808E0000E020168
:10234C005E1902E1000E5D1901E1A5D710EC0DF04C
:10235C00120E0301A66F3D0EA76F000EA86FC5EC01
:10236C000AF08FEC0CF08B0E0301A06F400EA16FE6
:10237C00000EA26F72EC0CF00D0E0301A66F5CEC5C
:10238C000AF01F0E0B6E710E0C6E1E0E0D6E0D2EC6
:10239C00FED70C2EFCD70B2EFAD70000000E020134
:1023AC00411902E1000E40190EE1000E5E1902E126
:1023BC00000E5D1908E1000E01013D5D02E1030E06
:1023CC003C5D01E2EBD7400E0301A06F010EA16F43
:1023DC003E0EA26F000EA36F030EA46F000EA56F2E
:1023EC00CDEC0CF0000E011802E1000E001808E014
:1023FC00000E02015E1902E1000E5D1901E1B1D778
:10240C0010EC0DF0BD0E0301A66F3E0EA76F000E73
:10241C00A86FC5EC0AF08FEC0CF0FC0E0301A06F5A
:10242C00400EA16F000EA26F72EC0CF00D0E0301AA
:10243C00A66F5CEC0AF01F0E0B6E710E0C6E1E0E6E
:10244C000D6E0D2EFED70C2EFCD70B2EFAD70000DE
:10245C00000E0201411902E1000E40190EE1000EBE
:10246C005E1902E1000E5D1908E1000E01013D5DEF
:10247C0002E1030E3C5D01E2EBD7400E0301A06FBD
:10248C00010EA16F3A0EA26F000EA36F030EA46F84
:10249C00000EA56FCDEC0CF0000E011802E1000E41
:1024AC00001808E0000E02015E1902E1000E5D1931
:1024BC0001E1B1D710EC0DF0C20E0301A66F3D0E79
:1024CC00A76F000EA86FC5EC0AF08FEC0CF0040E91
:1024DC000301A06F410EA16F000EA26F72EC0CF005
:1024EC000D0E0301A66F5CEC0AF01F0E0B6E710E45
:1024FC000C6E1E0E0D6E0D2EFED70C2EFCD70B2E59
:10250C00FAD70000000E0201411902E1000E401939
:10251C000EE1000E5E1902E1000E5D1908E1000EDD
:10252C0001013D5D02E1030E3C5D01E2EBD7400E83
:10253C000301A06F010EA16F420EA26F000EA36FDC
:10254C00030EA46F000EA56FCDEC0CF0000E01185D
:10255C0002E1000E001808E0000E02015E1902E113
:10256C00000E5D1901E1B1D710EC0DF0010E030165
:10257C00A66F400EA76F000EA86FC5EC0AF08FEC8B
:10258C000CF0120E0301A06F410EA16F000EA26F92
:10259C0072EC0CF00D0E0301A66F5CEC0AF01F0E32
:1025AC000B6E710E0C6E1E0E0D6E0D2EFED70C2EBC
:1025BC00FCD70B2EFAD70000000E0201411902E1E4
:1025CC00000E40190EE1000E5E1902E1000E5D19BD
:1025DC0008E1000E01013D5D02E1030E3C5D01E2EC
:1025EC00EBD7400E0301A06F010EA16F4A0EA26F34
:1025FC00000EA36F030EA46F000EA56FCDEC0CF0B4
:10260C00000E011802E1000E001808E0000E020195
:10261C005E1902E1000E5D1901E1B1D710EC0DF06D
:10262C00930E0301A66F3C0EA76F000EA86FC5ECAE
:10263C000AF08FEC0CF01C0E0301A06F410EA16F81
:10264C00000EA26F72EC0CF00D0E0301A66F5CEC89
:10265C000AF01F0E0B6E710E0C6E1E0E0D6E0D2EF3
:10266C00FED70C2EFCD70B2EFAD70000000E020161
:10267C00411902E1000E40190EE1000E5E1902E153
:10268C00000E5D1908E1000E01013D5D02E1030E33
:10269C003C5D01E2EBD7400E0301A06F010EA16F70
:1026AC00460EA26F000EA36F030EA46F000EA56F53
:1026BC00CDEC0CF0000E011802E1000E001808E041
:1026CC00000E02015E1902E1000E5D1901E1B1D7A5
:1026DC0010EC0DF081B20AD0D30E0301A66F3C0EA4
:1026EC00A76F000EA86FC5EC0AF009D08A0E030183
:1026FC00A66F3D0EA76F000EA86FC5EC0AF08FEC0D
:10270C000CF081B220D0F10E0301A06F3F0EA16F2F
:10271C00000EA26F72EC0CF00D0E0301A66F5CECB8
:10272C000AF0020E0301A66F000EA76F010EA86F30
:10273C00000EA96F160EAA6F3F0EAB6F000EAC6F9A
:10274C0095EC0BF01FD0E10E0301A06F3F0EA16FB3
:10275C00000EA26F72EC0CF00D0E0301A66F5CEC78
:10276C000AF0020E0301A66F000EA76F010EA86FF0
:10277C00000EA96FF40EAA6F3E0EAB6F000EAC6F7D
:10278C0095EC0BF01F0E0B6E710E0C6E1E0E0D6E7B
:10279C000D2EFED70C2EFCD70B2EFAD70000000EF8
:1027AC000201411902E1000E40190EE1000E5E1902
:1027BC0002E1000E5D1908E1000E01013D5D02E130
:1027CC00030E3C5D01E2EBD7400E0301A06F010E3E
:1027DC00A16F2E0EA26F000EA36F030EA46F000E3E
:1027EC00A56FCDEC0CF0000E011802E1000E0018E4
:1027FC0008E0000E02015E1902E1000E5D1901E114
:10280C007ED710EC0DF0320E01013E6F000E3F6FC3
:10281C00970E0301A66F3E0EA76F000EA86FC5ECB6
:10282C000AF08FEC0CF0210E0301A06F410EA16F8A
:10283C00000EA26F72EC0CF00D0E0301A66F5CEC97
:10284C000AF0040E0B6E0C0E0C6E330E0D6E0D2E6C
:10285C00FED70C2EFCD70B2EFAD700000000000E72
:10286C000201411902E1000E40190EE1000E5E1941
:10287C0002E1000E5D1908E1000E01013D5D02E16F
:10288C00030E3C5D01E2EBD7400E0301A06F010E7D
:10289C00A16F320EA26F000EA36F030EA46F000E79
:1028AC00A56FCDEC0CF0000E011802E1000E001823
:1028BC0008E0000E02015E1902E1000E5D1901E153
:1028CC00B0D710EC0DF03D0E0B6EE10E0C6E3F0E02
:1028DC000D6E0D2EFED70C2EFCD70B2EFAD700004A
:1028EC0000000A0E0301A66F3C0EA76F000EA86F26
:1028FC00C5EC0AF08FEC0CF0640E01013E6F000E7B
:10290C003F6F26EC09F0330E0301A06F410EA16F4F
:10291C00000EA26F72EC0CF00D0E0301A66F5CECB6
:10292C000AF0000E0201411902E1000E401907E104
:10293C00000E5E1902E1000E5D1901E1F2D7400EA6
:10294C000301A66F010EA76F42EC0AF037EC0BF0F7
:10295C00F30E0301A66F3C0EA76F000EA86FC5EC1B
:10296C000AF08FEC0CF0640E01013E6F000E3F6F0D
:10297C0026EC09F0350E0301A06F410EA16F000E7D
:10298C00A26F72EC0CF00D0E0301A66F5CEC0AF05A
:10299C00000E0201411902E1000E401907E1000E80
:1029AC005E1902E1000E5D1901E1F2D7400E030140
:1029BC00A66F010EA76F42EC0AF037EC0BF0320E4B
:1029CC0001013E6F000E3F6F26EC09F0F80E03017B
:1029DC00A66F3D0EA76F000EA86FC5EC0AF08FEC2A
:1029EC000CF02B0E0301A06F410EA16F000EA26F15
:1029FC0072EC0CF00D0E0301A66F5CEC0AF01F0ECE
:102A0C000B6E710E0C6E1E0E0D6E0D2EFED70C2E57
:102A1C00FCD70B2EFAD70000000E0201411902E17F
:102A2C00000E40190EE1000E5E1902E1000E5D1958
:102A3C0008E1000E01013D5D02E1030E3C5D01E287
:102A4C00EBD7400E0301A06F010EA16F360EA26FE3
:102A5C00000EA36F030EA46F000EA56FCDEC0CF04F
:102A6C00000E011802E1000E001808E0000E020131
:102A7C005E1902E1000E5D1901E1B1D710EC0DF009
:0A2A8C0052C200F053C201F0120024
:102A9600D10E0301A66F3F0EA76F000EA86FC5ECFF
:102AA6000AF095C3A0F3970E0301A16F030EA26F60
:102AB60038EC0CF0970EA66F030EA76F42EC0AF0E7
:102AC600F40EA66F400EA76F000EA86FC5EC0AF0B5
:102AD600D90E0301A66F400EA76F000EA86FC5ECB6
:102AE6000AF060EC08F095C3C4F383EC08F000C06C
:102AF60096F30050000A0CE0490E0301A66F400E43
:102B0600A76F000EA86FC5EC0AF00301966B0CD0F8
:102B16000301CF0EA66F400EA76F000EA86FC5EC7F
:102B26000AF0010E0301966F81EC08F037EC0BF00A
:062B360096C300F012003E
:102B3C00150E7B6E9F0E7A6E02015D6B5E6B799249
:102B4C00798A7988799C79967994798E7990A29200
:062B5C00A192A0921200FC
:102B6200C29EC29CC29AC298C296C284C280FF0E02
:102B7200C16EC192C18EC19CC18AC188C196C182F7
:062B8200C194C190120095
:102B8800020E0301A66F000EA76FE1EC09F0010E1B
:0E2B98000301A66F000EA76FE1EC09F012001A
:102BA6000301976B986B1F0E0B6E710E0C6E1E0E4B
:102BB6000D6E0D2EFED70C2EFCD70B2EFAD700006D
:102BC60060EC08F08DC3C4F383EC08F000C095F305
:102BD600000E0301966F000E961902E1000E95197C
:102BE60005E097C300F098C301F0E0D0974B982B0F
:102BF6000D0E0B6E2D0E0C6ED70E0D6E0D2EFED716
:102C06000C2EFCD70B2EFAD700000000C46B83EC09
:102C160008F000C095F3000E0301966F800E006E5B
:102C2600800E9619005C02E19551000805E297C3F3
:102C360000F098C301F0BAD0974B982B240EC46FBE
:102C460083EC08F00C0E0301C46F83EC08F0060E4B
:102C56000301C46F83EC08F0250E0301C46F83ECF7
:102C660008F0060E0301C46F83EC08F0110E030191
:102C7600C46F83EC08F0420E0301C46F83EC08F0C6
:102C8600960E0301C46F83EC08F0240E0301C46F93
:102C960083EC08F000C095F3000E0301966F800EDA
:102CA600006E800E9619005C02E19551000805E25F
:102CB60097C300F098C301F079D0974B982B0C0E70
:102CC600C46F83EC08F000C095F3000E0301966F05
:102CD600800E006E800E9619005C02E19551000888
:102CE60005E297C300F098C301F060D0974B982B8C
:102CF600060EC46F83EC08F000C095F3000E0301C6
:102D0600966F800E006E800E9619005C02E195515A
:102D1600000805E297C300F098C301F047D0974B2F
:102D2600982B020EC46F83EC08F000C095F3000EDA
:102D36000301966F800E006E800E9619005C02E10C
:102D46009551000805E297C300F098C301F02ED014
:102D5600974B982B010EC46F83EC08F000C095F3D7
:102D6600000E0301966F800E006E800E9619005CB1
:102D760002E19551000805E297C300F098C301F0FF
:102D860015D0070E0B6E170E0C6E6A0E0D6E0D2EFD
:102D9600FED70C2EFCD70B2EFAD7000081EC08F0DC
:0E2DA600974B982B97C300F098C301F01200D2
:102DB40000C023F001C022F002C021F003C020F0C3
:102DC40004C01FF005C01EF008C01DF009C01CF0AF
:102DD4000AC01BF00BC01AF0E1CF2CF0E2CF2DF0AB
:102DE400E9CF2AF0EACF2BF0F3CF28F0F4CF29F083
:102DF400F5CF27F0F8CF24F0F7CF25F0F6CF26F063
:102E04009EAA48D09DAA46D0ACA203D0AC98AC8868
:102E1400AC92ACA402D0AFCF79F2AFCF79F2020179
:102E240079510D0A08E0010E03018A5D02E1000EEA
:102E3400895D01E220D00301010E8B6F000E8C6FBF
:102E4400010E8A5D02E1000E895D04E3020E8B6FC0
:102E5400000E8C6FA09A7E0E8925E16E020E8A21E7
:102E6400E26EE66A89C387F38AC388F3896B8A6B47
:102E74000201796B0FD07E0E03018925E16E020EEB
:102E84008A21E26E79C2E6FF89C387F38AC388F395
:102E9400894B8A2BA4AA3FD0A3AA3DD09CA202D0DE
:102EA4009C989C889CA402D0AACF78F0AACF78F0F2
:102EB400000E00016C5D02E1FF0E6B5D08E25250F2
:102EC4000D0A04E178510D0A01E101D015D0A39A4D
:102ED400400E6B25E16E010E6C21E26EE66A6BC05A
:102EE4003CF16CC03DF16B6B6C6B786B010E0201B5
:102EF400406F000E416F0FD0400E00016B25E16E54
:102F0400010E6C21E26E78C0E6FF6BC03CF16CC030
:102F14003DF16B4B6C2B60EC0EF027C0F5FF24C029
:102F2400F8FF25C0F7FF26C0F6FF28C0F3FF29C02D
:102F3400F4FF23C000F022C001F021C002F020C041
:102F440003F01FC004F01EC005F01DC008F01CC033
:102F540009F01BC00AF01AC00BF02AC0E9FF2BC00D
:0C2F6400EAFF2CC0E1FF2DC0E2FF1100CD
:102F70009CEC20F0D38CD38AD388D382D3909B6AE5
:102F80009B8CD3B601D0FDD7D2EC0FF064EC0FF0E0
:102F90008C94140E01013E6F000E3F6F920E3A6F3B
:102FA000000E3B6F0001926B0101126B000E0301DA
:102FB000956F050E966F400E976F050E986F1BEC80
:102FC0000EF0020E0A6E310E0B6E620E0C6E450E86
:102FD0000D6E0D2EFED70C2EFCD70B2EFAD70A2E17
:102FE000F8D77E86010E7F6E370EB06EAD8499ECF9
:102FF0000DF00C0E0301C46FAAEC06F01F0E0B6E51
:10300000710E0C6E1E0E0D6E0D2EFED70C2EFCD703
:103010000B2EFAD70000640E0301A66F3B0EA76FBC
:10302000000EA86FC5EC0AF0100E0301A66F3A0E51
:10303000A76F000EA86FC5EC0AF04F0E0301A66F34
:103040003A0EA76F000EA86FC5EC0AF0BE0E030182
:10305000A66F3B0EA76F000EA86FC5EC0AF0FC0E22
:103060000301A66F3A0EA76F000EA86FC5EC0AF019
:10307000300E0301A66F3D0EA76F000EA86FC5ECC2
:103080000AF0D00E0301A66F390EA76F000EA86FCD
:10309000C5EC0AF0320E0301A66F3B0EA76F000EBF
:1030A000A86FC5EC0AF00D0E0B6E2D0E0C6ED70E30
:1030B0000D6E0D2EFED70C2EFCD70B2EFAD700006E
:1030C00000007C86020E7D6E700EAB6EA884EEEC66
:1030D0000DF00C0E0301A66F5CEC0AF01F0E0B6ED8
:1030E000710E0C6E1E0E0D6E0D2EFED70C2EFCD723
:1030F0000B2EFAD700000D0E0B6E2D0E0C6ED70E98
:103100000D6E0D2EFED70C2EFCD70B2EFAD700001D
:103110000000EBEC0FF0710EA66F400EA76F000ED3
:10312000A86FC5EC0AF0780E6E6E32EC0EF0A60EAB
:103130000301A66F3D0EA76F000EA86FC5EC0AF045
:10314000640E01013E6F000E3F6FF8DC740E030148
:103150008D6F740E0001846F100E736F2D0E0301BE
:10316000A66F3C0EA76F000EA86FC5EC0AF084C0D6
:1031700095F391DC00C090F0000E0001916F37ECE8
:103180000BF0460E0301A66F3E0EA76F000EA86F50
:10319000C5EC0AF008DD00C090F001C091F00A0E05
:1031A0000B6E220E0C6EA10E0D6E0D2EFED70C2E88
:1031B000FCD70B2EFAD7E8DC0A0E0B6E220E0C6E33
:1031C000A10E0D6E0D2EFED70C2EFCD70B2EFAD7AE
:1031D000010E0301A66F000EA76F010EA86F000E6F
:1031E000A96F7C0EAA6F3F0EAB6F000EAC6F95EC13
:1031F0000BF0020E0301A66F000EA76F010EA86F61
:10320000000EA96F8D0EAA6F3F0EAB6F000EAC6F54
:1032100095EC0BF07A0E0B6EC10E0C6E810E0D6EDE
:103220000D2EFED70C2EFCD70B2EFAD70000000077
:1032300098DC020E0301A66F000EA76F010EA86FA7
:10324000000EA96F9E0EAA6F3F0EAB6F000EAC6F03
:1032500095EC0BF07A0E0B6EC10E0C6E810E0D6E9E
:103260000D2EFED70C2EFCD70B2EFAD70000000037
:103270006F0E0301A66F3E0EA76F000EA86FC5EC80
:103280000AF0020E0301A66F000EA76FE1EC09F031
:10329000010E0301A66F000EA76F010EA86F000EAE
:1032A000A96F490EAA6F3F0EAB6F000EAC6F95EC85
:1032B0000BF03D0E0B6EE10E0C6E3F0E0D6E0D2EE3
:1032C000FED70C2EFCD70B2EFAD7000000004E0EB6
:1032D0000301A66F3D0EA76F000EA86FC5EC0AF0A4
:1032E000400E0301C46F050EC56FEB0EC66F400E96
:1032F000C76F000EC86F94EC08F0400E0301A06F7A
:10330000050EA16F400EA26F2DEC0CF0005201E1F2
:10331000F4D7DBEC10F0400E0301C46F050EC56F4F
:1033200053C0C6F354C0C7F355C0C8F394EC08F0BB
:10333000400E0301A06F050EA16F400EA26F2DEC91
:103340000CF0005201E1F4D7400E0301C46F050EEA
:10335000C56F56C0C6F357C0C7F358C0C8F394EC46
:1033600008F0400E0301A06F050EA16F400EA26F82
:103370002DEC0CF0005201E1F4D7070E0B6E170E86
:103380000C6E6A0E0D6E0D2EFED70C2EFCD70B2E7A
:10339000FAD70000DBEC10F02D0E0301A66F3E0EF5
:1033A000A76F000EA86FC5EC0AF0EBEC0FF08FECE6
:1033B0000CF08C94020E0301A66F000EA76FE1ECD7
:1033C00009F0010E0301A66F000EA76F010EA86F92
:1033D000000EA96F5A0EAA6F3F0EAB6F000EAC6FB6
:1033E00095EC0BF05C0E0B6E510E0C6E600E0D6EBC
:1033F0000D2EFED70C2EFCD70B2EFAD700009D8A7F
:10340000A38AF28CF28ED08E00018D6B8E6B526A85
:103410008C840D0E0B6E2D0E0C6ED70E0D6E0D2EB8
:10342000FED70C2EFCD70B2EFAD7000000008C9490
:103430000D0E0B6E2D0E0C6ED70E0D6E0D2EFED7D3
:103440000C2EFCD70B2EFAD7000000008C840D0E3A
:103450000B6E2D0E0C6ED70E0D6E0D2EFED70C2E94
:10346000FCD70B2EFAD700000000EEEC10F000C0E5
:1034700090F001C091F06C0E0301A66F3D0EA76F96
:10348000000EA86FC5EC0AF090C095F391C096F3BA
:10349000120E0301976F010E986F1DEC10F0120EC3
:1034A000A66F010EA76F42EC0AF0000E0001911901
:1034B00002E1090E90190AE1BA0E0301A66F400E4F
:1034C000A76F000EA86FC5EC0AF009D0AA0E030181
:1034D000A66F3E0EA76F000EA86FC5EC0AF037EC82
:1034E0000BF0020E0301A66F000EA76FE1EC09F0CE
:1034F000000E0001911902E1090E901912E1020E6D
:103500000301A66F000EA76F010EA86F000EA96F32
:103510006B0EAA6F3F0EAB6F000EAC6F95EC0BF00D
:1035200011D0020E0301A66F000EA76F010EA86F47
:10353000000EA96FAF0EAA6F3F0EAB6F000EAC6FFF
:1035400095EC0BF07A0E0B6EC10E0C6E810E0D6EAB
:103550000D2EFED70C2EFCD70B2EFAD70000000044
:103560000D0E526E640E01013E6F000E3F6F26EC91
:1035700009F0920E01013A6F000E3B6F3AC1C4F39D
:103580003BC1C5F3130E0301C66F3E0EC76F000E9D
:10359000C86F94EC08F0040E01013A25E16E000EAC
:1035A0003B21E26E006A83BE002A300E002600C076
:1035B000E6FF0D0E3A25E16E000E3B21E26E006A39
:1035C00087B6002A300E002600C0E6FF010E030178
:1035D000956F3DEC0EF000C086F001C087F000C092
:1035E00095F301C096F3120E0301976F010E986FC9
:1035F0001DEC10F03AC195F33BC196F3120E976F94
:10360000010E986FA2EC0FF03AC1A6F33BC1A7F3ED
:1036100042EC0AF037EC0BF03AC195F33BC196F35C
:1036200002EC10F00D0EA66F5CEC0AF08FEC0CF0C3
:10363000C4EC15F03AC1C4F33BC1C5F3AF0E0301AE
:10364000C66F400EC76F000EC86F94EC08F0030EF3
:1036500001013A25E16E000E3B21E26E006A83BE55
:10366000002A300E002600C0E6FF080E3A25E16E63
:10367000000E3B21E26E006A87B6002A300E00265B
:1036800000C0E6FF3AC195F33BC196F3120E030169
:10369000976F010E986FA2EC0FF0010EA66F000E4F
:1036A000A76F010EA86F000EA96F3AC1AAF33BC124
:1036B000ABF363EC0AF0020E0301A66F000EA76FD6
:1036C000010EA86F000EA96FC00EAA6F3F0EAB6F60
:1036D000000EAC6F95EC0BF05C0E0B6E510E0C6E89
:1036E000600E0D6E0D2EFED70C2EFCD70B2EFAD7CA
:1036F0000000000E02015E1902E1000E5D1907E1F3
:10370000000E411902E1010E401901E1F2D7000E4D
:10371000411902E1010E4019D8A48CD0100E03010A
:10372000A66F400EA76F000EA86FC5EC0AF0400E02
:103730000301A66F010EA76F42EC0AF037EC0BF005
:10374000C4EC15F0420E0301C46F020EC56FE20E09
:10375000C66F3E0EC76F000EC86F94EC08F0420EA5
:103760000301956F020E966F400E976F010E986FD2
:10377000090E996F000E9A6FC6EC0DF0120E956F40
:10378000010E966F4A0E976F010E986F100E996F8B
:10379000000E9A6F66EC10F0010EA66F000EA76F78
:1037A000010EA86F000EA96F120EAA6F010EAB6F6B
:1037B00063EC0AF0120E0301956F010E966F5A0E1C
:1037C000976F010E986F100E996F000E9A6F66EC4E
:1037D00010F0020EA66F000EA76F010EA86F000E6C
:1037E000A96F120EAA6F010EAB6F63EC0AF02D0EDB
:1037F0000301A66F400EA76F000EA86FC5EC0AF07C
:10380000420E0301A66F020EA76F42EC0AF037ECDE
:103810000BF05C0E0B6E510E0C6E600E0D6E0D2ECD
:10382000FED70C2EFCD70B2EFAD700008FEC0CF035
:10383000EBEC0FF00301000E8C1902E1010E8B1965
:103840006DE18FEC0CF01F0E0301A66F400EA76F09
:10385000000EA86FC5EC0AF07E0E0301A66F020EE3
:10386000A76F42EC0AF037EC0BF0C4EC15F0120E27
:103870000301956F010E966F880E976F020E986F79
:10388000100E996F000E9A6F66EC10F0010EA66F85
:10389000000EA76F010EA86F000EA96F3B0EAA6F56
:1038A000400EAB6F000EAC6F95EC0BF0020E0301F7
:1038B000A66F000EA76F010EA86F000EA96F120E63
:1038C000AA6F010EAB6F63EC0AF03D0E0B6EE10EBA
:1038D0000C6E3F0E0D6E0D2EFED70C2EFCD70B2E50
:1038E000FAD7000000007E0E0301956F020E966F5E
:1038F000620E976F000E986F040E996FAAEC10F08D
:10390000005001100BE0820E0301956F020E966FBE
:1039100002EC10F0EBEC0FF08FEC0CF023D6FFD79D
:1039200000C019F001C018F0156ED8CF16F0E0CF26
:1039300017F0A0A21FD0A1A21DD0010E01013E5D73
:10394000006E000E3F59016E00C03EF101C03FF114
:10395000000E3F1902E1000E3E190BE1010E0201BB
:103960005D6F000E5E6F7990150E7B6E9F0E7A6E06
:10397000A092A1921750E06E1650D86E153A1538E5
:0A39800019C000F018C001F010009B
:1041380010EE2EF0390E006E010E016E8A0EF66E2C
:0E4148003A0EF76E000EF86E58EC0EF01200F4
:10398A0050726F6A6574203A20436C69636B657282
:10399A00325F31384638374A35305F524E34315FFC
:1039AA0042545F6D61697472655F65745F47505315
:1039BA005F416E64726F69645F323031362E6D63B7
:0639CA007070690D0A0097
:1039D00020554152543220313932303020626473E4
:1039E00020436C69636B657232204D696B726F4264
:1039F0007573233120203C2D3E20426C7565546F39
:103A00006F7468436C69636B20524E34310D0A0049
:103A1000204469726563746F7279203A433A5F4D4E
:103A2000696B726F435F4D657350726F6A65747333
:103A30005F4D696B726F435F31384638374A3530B6
:0F3A40005F524E34315F4D61697472650D0A003B
:103A4F0020536F75726365204D696B726F4320430E
:103A5F006C69636B6572325F31384638374A35307F
:103A6F005F524E34315F42545F6D61697472655FAE
:0B3A7F003136303732302E630D0A0064
:043A8A00414F4B005D
:043A8E00414F4B0059
:043A9200454E440059
:043A9600414F4B0051
:043A9A00414F4B004D
:043A9E00414F4B0049
:043AA200414F4B0045
:043AA600414F4B0041
:043AAA00434D440044
:013AAE000017
:0F3AAF008A3900DD3D00E43B00C33A005B3E0076
:053ABE004364653D00BA
:103AC30031384638374A3530203A20546573747399
:103AD3002049542055415254312C55415254322CD3
:103AE30054696D6572302C41444330202620425482
:093AF30020524E34310D0A20006E
:103AFC0020554152543120333834303020626473B5
:103B0C0020436C69636B657232204D696B726F6216
:103B1C007573233220203C2D3E207465726D696EC6
:063B2C00616C200D0A008F
:103B3200204F7074696F6E6E656C3A205458205530
:103B42004152543320736F667420617420333834C9
:103B52003030206264732073757220524132200D1E
:023B62000A0057
:103B64002048617264776172653A20436C69636BC3
:103B74006572322031384638374A3530202B20429E
:103B84006C7565546F6F746820436C69636B0D0AC0
:013B94000030
:103B95000902290001010080320904000002030026
:103BA50000000921010100012221000705810340D0
:093BB500000107050103400001B5
:103BBE0020464F53433D384D687A20696E746572C6
:103BCE006E65207820504C4C203D3E2034384D6898
:063BDE007A20200D0A0010
:103BE4005541525420434F4D313A31393230302C03
:103BF40020554152543220434F4D32203A3139320C
:063C04003030200D0A0023
:103C0A00452020203D3E6469706C61792065787496
:103C1A00656E6465642073657474696E67203A2002
:033C2A000D0A0080
:103C2D00436865636B2070726573656E6365204CC8
:103C3D00434432313139206174204020307837349B
:033C4D000D0A005D
:103C500022034D0069006B0072006F0065006C006C
:103C600065006B00740072006F006E0069006B00ED
:023C70006100F1
:103C72000600FF0901A10119012940150026FF00D4
:103C820075089540810219012940750895409102F5
:013C9200C071
:103C930053412C30202064697361626C6520617527
:103CA3007468656E74696669636174696F6E0D002B
:103CB30020035500530042005F0052004E002D00C8
:103CC300340031005F0043006C00690063006B0047
:103CD30053522C3443304233413842393435372040
:103CE3003D3E2053746172616469637449490D00F8
:103CF3004F20203D3E20646973706C6179206F749E
:0F3D03006865722073657474696E67730D0A00CA
:103D1200534E2C4D7942542D44423439203D3E209D
:0E3D2200446576696365206E616D650D0A006B
:103D3000204C696169736F6E204D6F64656C6520FE
:0E3D4000425420524E343120617665632000DB
:103D4E0020417474656E746520696E6974204849EB
:0E3D5E0044207465726D696E616C200D0A0060
:103D6C00726573756C742042545F436F6E6669673D
:0E3D7C007572652829205374617465203D001E
:103D8A0053522C30303135383332423644383720AA
:0C3D9A003D3E2050435F41504D200D0085
:103DA600496E6974204932433220486172647761F2
:0C3DB6007265203430304B687A0D0A0032
:103DC20053542C323535203D3E20416C6C7761795D
:0B3DD2007320415420636465730D00F2
:103DDD00464F53433D34384D485A2020504C4C20CB
:0B3DED0061637469766520200D0A00F8
:103DF8002D2D2D2020203D3E2046696E206D6F64BC
:0B3E080065206364652041540D0A0032
:103E13004250313D202020203B4250323D20202083
:0A3E230020203B204541313D2000E6
:103E2D002041726D65204954205541525431202650
:093E3D002055415254320D0A00D7
:103E4600496E6974204C434420323131392032782E
:053E560031360D0A00E9
:103E5B00504F52542055534220434F4D2048494414
:043E6B00200D0A001C
:103E6F0020496E6974204849442055534220636F9E
:043E7F006D0D0A00BB
:103E83002424240D20204154204D6F646520456E69
:043E930074657200E0
:103E970053582C3120203D3E20426F6E6465643DAF
:033EA700310D00DA
:103EAA00202F2039202050726F626C656D6F20219F
:033EBA000D0A00EE
:103EBD0053552C31392E32203D3E2062617564738D
:033ECD000D0A00DB
:103ED000120100020000000834120100010001027A
:023EE0000001DF
:103EE20020202020202020202020202020202020D0
:023EF2002000AE
:103EF400546F2050435F585020636C652041504DEF
:013F040000BC
:103F0500425420436F6E66696775726174696F6E9E
:013F150000AB
:103F160020546F2053746172416469637449492067
:013F2600009A
:103F27004574617065203A202E2073757220392000
:013F37000089
:103F38004574617065203A203020737572203820EE
:013F48000078
:103F4900417474656E746520484944205465726DE6
:013F59000067
:103F5A0041726D6520496E74657272757074732052
:013F6A000056
:103F6B00496E697420425420636F6D706C65746583
:013F7B000045
:103F7C00496E69742054696D6572332034306D5309
:013F8C000034
:103F8D00203130302078203430203D20347365636B
:013F9D000023
:103F9E00496E697420414443207375722045413146
:013FAE000012
:103FAF0042616420696E69742042542021212020CF
:013FBF000001
:103FC00057616974696E672047505320646174615A
:013FD00000F0
:103FD100436865636B204465766963652040200012
:103FE10053522C3030313538333242364438370071
:103FF10053522C344330423341384239343537003F
:0F400100534D2C35203D3E20414E590D2072006D
:0F4010005374617261646963744949203A2000F6
:0E401F0055415254312052656375203A2000FD
:0E402D004865757265204750533D203A2000CB
:0E403B0055415254312052656375203A2000E1
:0E404900206973206E6F7420666F756E6400C0
:0D40570030303135383332423644383700CE
:0D406400344330423341384239343537009F
:0D40710020496E697420414443310D0A005E
:0D407E00443839353246334646373130007C
:0D408B00534E2C4D7942542D4442343900DF
:0C409800537461726164696374494900EB
:0B40A4000D0A5374617465203D20007C
:0B40AF0042313D2E2042323D2E200009
:0B40BA00202F203920204F4B0D0A0062
:0A40C500627566666572323D2000E8
:0A40CF0020666F756E64204F4B00F1
:0940D900322020484152445700F6
:0940E200415243484F53343300AE
:0940EB003136303732300D0A0085
:0840F400206F6E2049324300E9
:0840FC0053552C31392E32001E
:0741040053542C3235350045
:07410B0050435F41504D00DD
:05411200534D2C3500A7
:054117002D2D2D0D000F
:05411C0053412C3000AE
:0541210053582C310091
:054126002D2D2D0D0000
:04412B002D2D2D0009
:04412F000403090478
:02413300450045
:024135004F0039
:020000040001F9
:06FFF800ACF7C2FFF8FFA8
:00000001FF
